:0600000000308A003928DF
:100008008C0003088301AD000408AE000A08AF00A5
:100018008A012608B0002708B1002808B20029087C
:10002800B6002A08B4002B08B5002C08B3008B19B9
:080038000B1C20288312B822E2
:100040000B1083123008A6003108A7003208A80060
:100050003608A9003408AA003508AB003308AC0004
:100060002E0884002F088A002D0883008C0E0C0EA9
:1000700009000D30840026304120292B0406800120
:10008000840A0406031D3E2864000034AC01AA0162
:10009000AB0128082904031D5028A601A70100343C
:1000A0001F30AC040310AC0AA80DA90D031C532883
:1000B000A90CA80C29082702031D6028280826027D
:1000C000031C68282808A6022908031C290AA7027D
:1000D000AA0DAB0DAC0BAC1A5828AC1F7428AA099A
:1000E000AA0A0319AB03AB092A08A8002B08A90028
:1000F0002C1F0034A609A60A0319A703A709003478
:100100008312A3000A30A400A50123088E000E0D5F
:100110000E0D0139A600260C031C90280615912807
:1001200006110E0EA600A60C260C0139A600260C00
:10013000031C9C2886159D2886110E0EA600260CF1
:100140000139A600260C031CA7288614A8288610AF
:100150000E0E0139A600260C031CB0280614B12887
:100160000610061606120E0CA600A60C260C013967
:10017000A600260C031CBE280615BF2806110E0C6F
:10018000A600260C0139A600260C031CC9288615DA
:10019000CA2886110E0C0139A600260C031CD22891
:1001A0008614D32886100E080139A600260C031CDD
:1001B000DB280614DC28061006160612240803198C
:1001C000A503A403240A0319250A03190800DE283D
:1001D0008312861280308312802086161508A000B4
:1001E0001608A100C321063080200F08A000A1013D
:1001F000C321110880201008802020308020463044
:1002000080204D308020203080201508A000160866
:10021000A100C3211408303A031D10292030940096
:100220001408802013088020120880202E3080209F
:1002300011088020100880204D3080204830802018
:100240007A3080201A30A800A9011608A7001508E6
:10025000A600F030A6070318A70ADD30A70746203E
:100260002A089E002B089F001E08D82238218029CA
:100270000530A800A90183121608A7001508A600DA
:100280002E30A6070318A70A0430A70746202A081D
:1002900098002B0899000514A00165292008A800E2
:1002A0001908A7001808A600A80A59290310A70CC6
:1002B000A60CA80B5629260C031C602905156129DC
:1002C00005118312A00A8312A7230E302002031CFB
:1002D0004E2905118312A7230511A7230511A72372
:1002E0000511A7230511A7230511A7230511A7238E
:1002F0000511A7230515A7230515A7230510080039
:10030000831688188029831289010F08880003103A
:100310008B1B03148B138316081555308900AA30E4
:1003200089008814081103188B17881895298312DF
:100330000F080F0789001608880003108B1B031491
:100340008B138316081555308900AA30890088144C
:10035000081103188B178818AB29031483120F0D8B
:1003600089001508880003108B1B03148B13831658
:10037000081555308900AA3089008814081103181F
:100380008B17831208003030831290009100920086
:1003900093009400D229940AF030A0070318A10A10
:1003A000D830A10727302102103003192002031C86
:1003B000E129CB29930A1830A0070318A10AFC30C1
:1003C000A10703302102E83003192002031CEE29A3
:1003D000DA29920A9C30A007031CA10300302102F5
:1003E000643003192002031CFB29E929910AF63025
:1003F000A007031CA103003021020A3003192002C8
:100400000318F62920089007080083128612773017
:10041000831280208616003080201F30802011300B
:100420008020113080201F308020043080200E304A
:100430008020153080209F019F0AA0012C2AA00A4D
:100440009E0108301E0203182A2A9E0A1F088312E2
:100450008020212A03109F0D05302002031C1F2A33
:1004600073309F00A0010530200203180800A00A85
:10047000F8309F0786121F088312802086161F30CF
:100480008020332A533083129C0005309D001C08C5
:1004900003199D039C031C0A03191D0A031D472A07
:1004A000861206118611861406100616061274307E
:1004B0009C0001309D001C0803199D039C031C0A2D
:1004C00003191D0A031D5B2A2B3083128020133071
:1004D00080200C308020043080200522132B8312D2
:1004E0000F080F0789008316081483120808960066
:1004F000950103140F0D8900831608148312080850
:1005000095070318960A2A3016023130031915028E
:100510000318912A2230160210300319150203180D
:100520000800103095002730960008008312F8224A
:10053000970803190800170B9E2A4F231708023A41
:10054000031960231708033A031980231708043A94
:1005500003197123FF309C002F309D001C080319E4
:100560009D039C031C0A03191D0A03190800AE2AE7
:1005700083128D10861B8D140D11061B0D150D1D7C
:10058000C32A0130C42A0030A6008D1DC92A0130BB
:10059000CA2A0030A606031D0D19D42A8D18D22AA6
:1005A0000D16D32A0D120D148D110D198D1508007D
:1005B0008312A0008612C030831280208616A2010A
:1005C000F32AA101053021020318F02AA20AA10A88
:1005D00020082206031DE22A210883128020E22A35
:1005E0002D30831280205030220203180800E12AA7
:1005F00083129701CF308316860083120618022BD0
:100600009701970A8618062B0230970006190A2BC5
:100610000330970086190E2B04309700C0308316E4
:10062000860083120800B53083129E009F01861257
:100630000130831280201E0803199F039E031E0AA7
:1006400003191F0A031D1B2B86128030802086167B
:100650000800FF3083129A009B001A0803199B03BD
:100660009A031A0A03191B0A031D2D2B83128F23C9
:1006700042223D23E820AD233B2B831289018316C0
:100680000814831208088F0015300F0203184C2B32
:1006900001300F0203186F2A8F018F0A6F2AFB3077
:1006A00083129507031C960322301602103003199B
:1006B00015020318E828303095002A309600E82803
:1006C0000530831295070318960A2A301602313036
:1006D00003191502031CE8281030950022309600FB
:1006E000E82883128F0A15300F02031C792B8F0123
:1006F0008F0A6F22E820970803190800F8227B2B45
:1007000083128F0301300F020318882B14308F00DF
:100710006F22E820970803190800F8228A2B8B0122
:1007200083168501C03086008312850186018316F9
:1007300081138B150B108B178312080083120D1C6D
:1007400008000D1A4F230D1E60230D10E82800002D
:100750008312851500008511080083129E23962AB6
:02400E00F13F80
:104200000100FF0027004C002700A6002700E20065
:104210002800140028006E002800BE002800F000CE
:10422000290022002200560022007E002200A60063
:1042300023008C002600F70027004C002700A60072
:104240002700E2002800140028006E002800BE00AD
:104250002800F000FF00FF00FF00FF00FF00FF004C
:00000001FF
